:1070000055C000008AC0000088C0000086C0000093
:1070100084C0000082C0000080C000007EC000006C
:107020007CC000007AC0000019C5000076C00000D6
:1070300074C0000072C0000070C000006EC000008C
:107040006CC000006AC0000068C0000066C000009C
:107050000AC3000062C0000060C000005EC0000003
:107060005CC000005AC0000058C0000056C00000BC
:1070700054C0000052C0000050C000004EC00000CC
:107080004CC000004AC0000048C0000046C00000DC
:1070900044C0000042C0000040C000003EC00000EC
:1070A0003CC000003AC0000038C0000011241FBEE0
:1070B000CFEFDAE0DEBFCDBF04B603FE19C080918A
:1070C000A0019091A10182349C4D91F484B7877FF7
:1070D00084BF88E10FB6F89480936000109260003E
:1070E0000FBE1092A1011092A001E0E0F0E009951E
:1070F00011E0A0E0B1E0E8E2FEE702C005900D92E9
:10710000A239B107D9F721E0A2E9B1E001C01D928F
:10711000A03AB207E1F731D085C672CF84E0809300
:10712000E9008091E80085FD0EC08091E8008B7732
:107130008093E8008091E80082FDF3CF8EB3811147
:10714000F9CF80E008958091F100089593E0909345
:10715000E9009091E80095FF03C08093F100089545
:107160009091E8009E779093E8009091E80090FD60
:10717000F4CF9EB39111F9CF0895CF93DF9300D050
:107180001F92CDB7DEB784B7877F84BF88E10FB683
:10719000F89480936000109260000FBE90E080E849
:1071A0000FB6F89480936100909361000FBE11E0D8
:1071B00015BF82E085BF35D410936F0083E08093C4
:1071C00081007894A3E07A2EB5E06B2E212C312C2F
:1071D00080910001882309F42FC284E08093E900A4
:1071E0008091E80082FF26C299DF982F853419F438
:1071F0001092000107C088E8890F823010F09435A2
:1072000021F48CDF8DE0A2DFEDC19035D9F39C3401
:10721000C9F3943721F484E499DF80E0F4CF913608
:1072200011F489E5F0CF913491F478DF082F76DFFF
:1072300090E0880F991F202F30E0322F2227330F44
:10724000822B932BAA2797FDA095BA2F9FC1903729
:1072500011F483E5D8CF933571F47AE8E72E71E025
:10726000F72EF70181917F0171DFF1E9EF16F1E06F
:10727000FF06B9F7B7C1963521F481E367DF80E3F4
:10728000C2CF933731F487E861DF85E95FDF8EE1B4
:10729000BACF9536A9F4E0E0F0E070925700E89597
:1072A00007B600FCFDCF60925700E89507B600FCDA
:1072B000FDCFE058FF4FE11580E7F80771F7A2CF47
:1072C0009C3651F42BDF809599E0E1E0F0E0082E48
:1072D00090935700E89596CF923721F489E0E1E04A
:1072E000F0E010C0963419F489E0F1010BC09E342F
:1072F00021F489E0E3E0F0E005C0913539F489E05C
:10730000E2E0F0E08093570084917DCF923631F433
:1073100089E51CDF80E01ADF80E875CF923419F030
:10732000973609F0CEC09983F9DEA82EB12CBA2C7D
:10733000AA24F4DEA82AF2DE082F8BEB800F9981B5
:10734000823010F08FE35FCF973609F044C081E1BF
:1073500080935700E8954501B12C8114910409F4FC
:1073600041C1C0909201D0909301E0909401F090BF
:1073700095010634B9F4EB2DF0E0EC29FD29849158
:10738000E5DEBB2069F0F2E0CF0ED11CE11CF11C60
:10739000C0929201D0929301E0929401F0929501F3
:1073A000B12615C0D701C601B695A79597958795C3
:1073B00023D5CCDE82E0C80ED11CE11CF11CC092AA
:1073C0009201D0929301E0929401F092950191E0A4
:1073D000891A9108C2CFC0909201D0909301E09099
:1073E0009401F0909501063429F0BB82AA82412CC9
:1073F000512C31C0F60170925700E89507B600FC99
:10740000FDCFF3CF063479F5552051F180909201EC
:1074100090909301A0909401B09095017FDE242D6F
:1074200030E0382BF401090110935700E89511243E
:10743000F2E08F0E911CA11CB11C809292019092DF
:107440009301A0929401B092950151268A819B816B
:1074500001979B838A83EA81FB81EF2B99F626C0F3
:107460005DDE482EF2CF5ADE682F80919201909116
:107470009301A0919401B0919501B695A795979528
:107480008795C2D48091920190919301A09194012B
:10749000B09195010296A11DB11D80939201909328
:1074A0009301A0939401B0939501D0CF063409F0D5
:1074B000A9CEF60160925700E89507B600FCFDCF13
:1074C000A1CE933469F4E0909201F090930126DE0E
:1074D00090E0F7010C0110935700E895112492CE2B
:1074E0009336F9F4C0909201D0909301E09094010A
:1074F000F090950113DEF601E16090E00C0110932D
:107500005700E8951124F2E0CF0ED11CE11CF11CCC
:10751000C0929201D0929301E0929401F092950171
:1075200071CE9D3659F4E0919201F09193016092F1
:107530005700E89507B600FCFDCF64CE923551F4B4
:10754000E0919201F0919301E590F4908F2DFEDD92
:107550008E2D59CE943419F5E1DD682F809192017A
:1075600090919301A0919401B0919501B695A79542
:107570009795879549D48091920190919301A0911C
:107580009401B09195010296A11DB11D80939201C5
:1075900090939301A0939401B093950133CE9436C8
:1075A000F1F4C0909201D0909301E0909401F0909A
:1075B0009501D701C601B695A795979587951CD4D7
:1075C000C5DD82E0C80ED11CE11CF11CC092920105
:1075D000D0929301E0929401F092950103C09B3107
:1075E00009F0B0CE7092E9009091E8008091E80037
:1075F0008E778093E80095FD11C08091E80080FDB2
:1076000004C08EB38111F9CF15C08091E8008E7748
:107610008093E80003C08EB3882361F08091E80076
:1076200080FFF9CF94E09093E9008091E8008B7798
:107630008093E800C6D3CCCD8091E0008160809338
:10764000E00082E49CED9093A1018093A0012CE0E6
:1076500088E190E00FB6F894A895809360000FBE83
:1076600020936000FFCF1F920F920FB60F9211244C
:107670000F900FBE0F901F90189542E061EC82E0D2
:1076800062D142E161E883E05ED142E160E884E0FA
:107690005AC180919801982F9F77913299F59091D6
:1076A0009901913229F0923229F1903259F510C0A6
:1076B000813A41F58091E800877F8093E80067E098
:1076C00070E081E091E0A4D08091E8008B770FC05A
:1076D0008132C1F48091E800877F8093E80067E001
:1076E00070E081E091E0F1D08091E8008E778093A6
:1076F000E8000895813231F48091E800877F80931B
:10770000E80035C10895292F30E02230310539F0E5
:107710002330310549F02130310561F410C08EE38A
:1077200090E02AE331E01EC0882371F0813089F0B7
:107730008230A1F080E090E020E030E013C082E1F0
:1077400090E028E731E00EC084E090E026E331E0ED
:1077500009C088E190E02CE131E004C082E190E0D2
:1077600028E031E0FA0131832083089507B600FC58
:10777000FDCFF999FECF23E0FB0120935700E89558
:1077800007B600FCFDCF81E180935700E89508958E
:1077900007B600FCFDCFF999FECF25E0FB01209351
:1077A0005700E89507B600FCFDCF81E180935700B4
:1077B000E895089507B600FCFDCFF999FECF21E0CA
:1077C000FB010A0120935700E8951124089521E256
:1077D000FC01209357008491089529E0FC01209337
:1077E000570084910895E1E0F0E089E0809357002C
:1077F0008491089507B600FCFDCFF999FECF8095DE
:1078000099E0E1E0F0E0082E90935700E8950895A4
:1078100020919E0130919F012617370748F061158E
:10782000710539F42091E8002E772093E80001C01B
:10783000B901FC0120E061157105A1F18EB3882327
:10784000F1F18530F1F18091E80083FD3CC0809139
:10785000E80082FF06C08091E80082FF26C080E039
:1078600008958091E80080FFE6CF2091F300809199
:10787000F20090E0922B6115710551F0883091056E
:1078800038F421912093F100615071090196F3CFF2
:1078900021E0089709F020E08091E8008E7780933E
:1078A000E800C9CF2111CACFD6CF8EB3882339F0D3
:1078B000853039F08091E80083FFCDCF04C082E0AD
:1078C000089583E0089581E008956115710529F414
:1078D0002091E8002B772093E8006115710531F1C4
:1078E0002EB3222361F1253061F12091E80023FDC0
:1078F00022C02091E80022FFF3CFFC01CF0140918C
:10790000F3002091F20030E0342B232B09F3809117
:10791000F1008193CF01615071096115710571F713
:10792000D7CF8EB3882359F0853059F08091E80085
:1079300080FFF7CF02C081E0089580E0089582E0E3
:10794000089583E008958F708093E900EBEEF0E0F6
:10795000808181608083EDEEF0E010826093EC0026
:1079600040838091EE00881F8827881F08958091AA
:10797000980187FD05C08091E80080FF0DC010C010
:107980008091E80082FD04C08EB38111F9CF089583
:107990008091E8008B7707C08EB38111ECCF0895FA
:1079A0008091E8008E778093E80008950F931F93ED
:1079B000CF93DF9346D04DD0C8EDD0E088818F774C
:1079C000888388818068888388818F7D888319BCBB
:1079D0001EBA1092960100EE10E0F80180818B7FB4
:1079E000808388818160888342E060E080E0ABDF53
:1079F000E1EEF0E080818E7F8083E2EEF0E0808136
:107A000081608083808188608083F80180818E7F9F
:107A10008083888180618883DF91CF911F910F914E
:107A20000895E8EDF0E080818F7E8083E7EDF0E05F
:107A300080818160808384E082BF81E080939701B0
:107A4000B5CFE8EDF0E080818E7F80831092E20078
:107A500008951092DA001092E10008951F920F929B
:107A60000FB60F9211242F933F934F935F936F9311
:107A70007F938F939F93AF93BF93EF93FF938091E7
:107A8000DA0080FF19C08091D80080FF15C0809176
:107A9000DA008E7F8093DA008091D90019BC80FFD4
:107AA00009C082E089BD09B400FEFDCF81E08EBB34
:107AB00087D102C01EBA84D18091E10080FF17C037
:107AC0008091E20080FF13C08091E2008E7F80935E
:107AD000E2008091E20080618093E2008091D80012
:107AE00080628093D80019BC85E08EBB69D18091FB
:107AF000E10084FF2DC08091E20084FF29C019BC01
:107B000082E089BD09B400FEFDCF8091D8008F7D51
:107B10008093D8008091E1008F7E8093E100809176
:107B2000E2008F7E8093E2008091E200816080938A
:107B3000E20080919601882311F084E007C08091D3
:107B4000E30087FF02C083E001C081E08EBB38D133
:107B50008091E10083FF21C08091E20083FF1DC07E
:107B60008091E100877F8093E10082E08EBB1092DC
:107B700096018091E1008E7F8093E1008091E20088
:107B80008E7F8093E2008091E20080618093E2002A
:107B900042E060E080E0D7DE13D1FF91EF91BF912A
:107BA000AF919F918F917F916F915F914F913F9195
:107BB0002F910F900FBE0F901F9018951F93CF938A
:107BC000DF9300D0CDB7DEB7E8E9F1E08091F100B6
:107BD000819381E0E03AF807C9F75BDD8091E80026
:107BE00083FFDAC09091980180919901853009F462
:107BF00065C030F4813059F168F0833041F1CCC078
:107C0000883009F49CC0893009F4ABC0863009F093
:107C1000C3C075C0903881F0923809F0BDC0809122
:107C20009C018F708093E9009091EB0095FB992760
:107C300090F91092E90001C090E08091E800877F00
:107C40008093E8009093F1001092F10083C0292FF7
:107C50002D7F09F0A1C0923009F09EC090919A0149
:107C6000911126C020919C012F7009F495C020939A
:107C7000E9009091EB0090FF1BC0833021F48091CC
:107C8000EB00806213C08091EB0080618093EB0079
:107C900081E090E0022E01C0880F0A94EAF78093F9
:107CA000EA001092EA008091EB0088608093EB007C
:107CB0001092E9008091E800877F4FC091116CC05D
:107CC00010919A011F778091E3008078812B809337
:107CD000E3008091E800877F8093E80048DE809190
:107CE000E80080FFFCCF8091E30080688093E30090
:107CF000112311F083E001C082E08EBB4DC090588B
:107D0000923008F049C0AE014F5F5F4F60919C0117
:107D100080919A0190919B01F6DC009709F43CC098
:107D20002091E800277F2093E800BC0189819A8197
:107D30006FDD8091E8008B778093E8002DC090384C
:107D400059F58091E800877F8093E8008091960143
:107D50008093F1008091E8008E778093E80007DE41
:107D60001BC0911119C090919A019230A8F4809192
:107D7000E800877F8093E80090939601F8DD80917A
:107D80009601811104C08091E30087FF02C084E066
:107D900001C081E08EBB71DC8091E80083FF0AC0E6
:107DA0008091E800877F8093E8008091EB008062FB
:107DB0008093EB000F900F90DF91CF911F9108956A
:107DC0000895CF938EB38823A9F08091E9008F7036
:107DD0009091EC0090FF02C090E801C090E0C92FA4
:107DE000C82B1092E9008091E80083FDE7DECF7098
:107DF000C093E900CF910895F999FECF92BD81BD5E
:107E0000F89A992780B50895262FF999FECF1FBAC1
:107E100092BD81BD20BD0FB6F894FA9AF99A0FBEB3
:087E200001960895F894FFCFCC
:107E2800010000000000000812034C005500460045
:107E380041002000430044004300000018034400B0
:107E4800650061006E002000430061006D00650060
:107E58007200610000000403090409023E000201E7
:107E6800008032090400000102020100052400100C
:107E78000104240202052406000107058203080004
:107E8800FF09040100020A000000070504021000AF
:107E98000507058302100005120110010200000801
:107EA800EB034A200001010200014C5546414344BE
:027EB800430085
:107FA000E5CBF6CB07CC13CC18CC1DCC23CC089555
:087FB000089508950895089555
:107FE000DFCFDFCFDFCFDFCFDFCFDFCFDFCFDFCF21
:087FF000DFCFDFCFDFCFDFCFD1
:087FF8000070000000DFFBDC5B
:040000030000700089
:00000001FF
